S0220000687474703A2F2F737265636F72642E736F75726365666F7267652E6E65742F1D
S12300000C9438000C94AD240C94E71D0C945F000C945F000C945F000C945F000C945F00F4
S12300200C945F000C9410270C945F000C94B52A0C945F000C94DB1E0C94A51E0C940C1DA4
S12300400C94B52B0C945F000C94342B0C945F000C94502C0C94182C0C945F000C945F0021
S12300600C945F000C945F000C945F000C945F0011241FBECFEFD0E1DEBFCDBF14BEA895C7
S123008088E10FB6F89480936000109260000FBE13E0A0E0B1E0EEE3FCE502C005900D92B4
S12300A0AA3EB107D9F718E0AAEEB3E001C01D92A835B107E1F70E94D0150C941D2E0C94BA
S12300C000009C01F999FECF32BD21BDF89A80B508959C01F999FECF1FBA32BD21BD60BD30
S12300E00FB6F894FA9AF99A0FBE089520E030E0F999FECF28593D4F32BD21BD28563240E1
S1230100F89A80B5F901E35DF94F80832F5F3F4F81E02034380761F720E030E0F999FECFB8
S123012028573E4F32BD21BD28583140F89A80B5F901E25CFE4F80832F5F3F4F25303105FB
S123014069F712BC11BC089580E090E0FC01E35DF94FE081F999FECF1FBA88599D4F92BDF9
S123016081BDE0BD0FB6F894FA9AF99A0FBE8756924021E08034920749F712BC11BC0895E6
S123018020E030E0F999FECF205F3F4F32BD21BD20513040F89A80B5F901E654FB4F8083E9
S12301A02F5F3F4F81E02034380761F712BC11BC089580E090E0FC01E654FB4FE081F99957
S12301C0FECF1FBA409692BD81BDE0BD0FB6F894FA9AF99A0FBE0F9721E08034920759F7EC
S12301E012BC11BC089520E430E0F999FECF205B3E4F32BD21BD20553140F89A80B5F901D4
S1230200EB5BFE4F80832F5F3F4F203A310569F712BC11BC089580E490E0FC01EB5BFE4F9C
S1230220E081F999FECF1FBA805B9E4F92BD81BDE0BD0FB6F894FA9AF99A0FBE8F54914036
S1230240803A910551F712BC11BC0895F999FECF82E090E092BD81BDF89A80B590E09093B2
S1230260200180931F0140911F0150912001F999FECF83E090E092BD81BDF89A20B5922F4C
S123028080E0840F951F9093200180931F01F999FECF8DEE93E092BD81BDF89A80B590E02B
S12302A090932401809323014091230150912401F999FECF8EEE93E092BD81BDF89A20B57E
S12302C0922F80E0840F951F909324018093230180911F0190912001909322018093210145
S12302E0F999FECF84E090E092BD81BDF89A80B590E09093260180932501409125015091A8
S12303002601F999FECF85E090E092BD81BDF89A20B5922F80E0840F951F909326018093C5
S12303202501F999FECF86E090E092BD81BDF89A80B590E09093010180930001409100018F
S123034050910101F999FECF87E090E092BD81BDF89A20B5922F80E0840F951F90930101FF
S123036080930001F999FECF81E090E092BD81BDF89A80B58093EA03F999FECF88E090E0AA
S123038092BD81BDF89A80B580931301F999FECF89E591E092BD81BDF89A80B580932F0109
S12303A0F999FECF82E094E092BD81BDF89A90B5892F8150853078F080912F01843039F4D8
S12303C081E08093180183E68093FF0506C082E08093180102C090931801F999FECF89E0F2
S12303E090E092BD81BDF89A80B580931201F999FECF84E094E092BD81BDF89A80B5809371
S1230400AE048091AE04823E24F08091AE048F3114F01092AE04F999FECF8EE090E092BD28
S123042081BDF89A80B580932801F999FECF8BE090E092BD81BDF89A80B520911801829FFE
S1230440C001112490931A0180931901F999FECF83E094E092BD81BDF89A80B580931B017E
S1230460F999FECF8CE090E092BD81BDF89A80B520911801829FC001112490931D018093B4
S12304801C01F999FECF8FE691E092BD81BDF89A80B580931E01F999FECF82EF91E092BDE0
S12304A081BDF89A80B580935F0480915F04882319F081E080935F04F999FECF8DE090E082
S12304C092BD81BDF89A80B526E0829FC00111249093150180931401F999FECF81E791E00E
S12304E092BD81BDF89A80B580932306F999FECF80E791E092BD81BDF89A80B580932106A3
S12305008AE08093920781E080939007F999FECF8FE891E092BD81BDF89A80B580933001D7
S12305208091300181FF05C080913001827F809330018091300185FF05C0809130018F72DB
S123054080933001F999FECF84EF91E092BD81BDF89A80B590E02CE231E0AC01429FC001DE
S1230560439F900D529F900D11249093B9048093B804F999FECF85EF91E092BD81BDF89A23
S123058080B58093B504F999FECF86EF91E092BD81BDF89A80B58093B304F999FECF87EF1E
S12305A091E092BD81BDF89A80B58093B204F999FECF88EF91E092BD81BDF89A80B590E09E
S12305C09093B1048093B0044091B0045091B104F999FECF89EF91E092BD81BDF89A20B521
S12305E0922F80E0840F951F9093B1048093B004F999FECF8BEF91E092BD81BDF89A80B552
S123060090E090933201809331014091310150913201F999FECF8CEF91E092BD81BDF89A4A
S123062020B5922F80E0840F951F9093320180933101F999FECF8DEF91E092BD81BDF89A73
S123064080B590E090933401809333014091330150913401F999FECF8EEF91E092BD81BD5D
S1230660F89A20B5922F80E0840F951F9093340180933301F999FECF8FEF91E092BD81BD2D
S1230680F89A80B590E090937803809377034091770350917803F999FECF80E092E092BDCD
S12306A081BDF89A20B5922F80E0840F951F909378038093770320E030E0F999FECF225A13
S12306C03E4F32BD21BD2E553140F89A80B5F901EB51FE4F8083F999FECF2E583E4F32BD1A
S12306E021BD22573140F89A80B5F901E050FA4F8083F999FECF24583E4F32BD21BD2C5739
S12307003140F89A80B5F901E050FA4F808B2F5F3F4F2A30310509F0D0CFF999FECF87E015
S123072092E092BD81BDF89A80B580933901F999FECF83E092E092BD81BDF89A80B5809307
S12307403A0120E030E094E6F901E159F84F908BF999FECF245E3D4F32BD21BD2C51324011
S1230760F89A80B5F901E159F84F80832F5F3F4F2031310549F720E030E0F999FECF27595E
S12307803E4F32BD21BD29563140F89A80B5F901E65DFE4F80832F5F3F4F2430310569F7B1
S12307A020E030E0F999FECF225D3D4F32BD21BD2E523240F89A80B5F901E454FC4F8083B5
S12307C02F5F3F4F2031310569F7F999FECF8DE691E092BD81BDF89A80B580932701F999AE
S12307E0FECF81EF91E092BD81BDF89A80B580935E04F999FECF80EF91E092BD81BDF89A20
S123080080B580932E01F999FECF86E092E092BD81BDF89A80B58093290120E030E0F999F3
S1230820FECF2A543C4F32BD21BD265B3340F89A80B5F901E151FE4F80832F5F3F4F20316D
S1230840310569F7F999FECF87EC93E092BD81BDF89A80B580933C01F999FECF88EC93E0CF
S123086092BD81BDF89A80B580933D01F999FECF84ED93E092BD81BDF89A80B580936A04B7
S1230880F999FECF85ED93E092BD81BDF89A80B580936B04F999FECF86ED93E092BD81BD68
S12308A0F89A80B580936C04F999FECF87ED93E092BD81BDF89A80B580936D04F999FECF6D
S12308C088EE93E092BD81BDF89A80B590E090933601809335014091350150913601F99913
S12308E0FECF89EE93E092BD81BDF89A20B5922F80E0840F951F9093360180933501F999AC
S1230900FECF8AEE93E092BD81BDF89A80B580936104F999FECF8CEC93E092BD81BDF89AE6
S123092080B52AE0829FC00111249093750480937404F999FECF81ED93E092BD81BDF89AD7
S123094080B52AE0829FC001112490937A0480937904F999FECF82ED93E092BD81BDF89AAC
S123096080B52AE0829FC001112490937C0480937B0412BC11BC089520911F0130912001FD
S1230980F999FECF1FBA82E090E092BD81BD20BD0FB6F894FA9AF99A0FBE20911F01309108
S12309A02001F999FECF1FBA83E090E092BD81BD30BD0FB6F894FA9AF99A0FBE2091250171
S12309C030912601F999FECF1FBA84E090E092BD81BD20BD0FB6F894FA9AF99A0FBE2091BF
S12309E0250130912601F999FECF1FBA85E090E092BD81BD30BD0FB6F894FA9AF99A0FBE19
S1230A002091000130910101F999FECF1FBA86E090E092BD81BD20BD0FB6F894FA9AF99A6D
S1230A200FBE2091000130910101F999FECF1FBA87E090E092BD81BD30BD0FB6F894FA9A02
S1230A40F99A0FBE20911301F999FECF1FBA88E090E092BD81BD20BD0FB6F894FA9AF99A7B
S1230A600FBE20911201F999FECF1FBA89E090E092BD81BD20BD0FB6F894FA9AF99A0FBE21
S1230A8012BC11BC0895F999FECF1FBA81EF91E092BD81BD10BC0FB6F894FA9AF99A0FBE63
S1230AA0F999FECF1FBA80EF91E092BD81BD8AE080BD0FB6F894FA9AF99A0FBE20915F048D
S1230AC0F999FECF1FBA82EF91E092BD81BD20BD0FB6F894FA9AF99A0FBEF999FECF1FBA11
S1230AE089E591E092BD81BD84E080BD0FB6F894FA9AF99A0FBEF999FECF1FBA8CE090E08C
S1230B0092BD81BD85E080BD0FB6F894FA9AF99A0FBEF999FECF1FBA8FE691E092BD81BDB2
S1230B2082E380BD0FB6F894FA9AF99A0FBEF999FECF1FBA81E791E092BD81BD84E180BD8A
S1230B400FB6F894FA9AF99A0FBEF999FECF1FBA80E791E092BD81BD81E080BD0FB6F894C0
S1230B60FA9AF99A0FBEF999FECF1FBA84EF91E092BD81BD88EC80BD0FB6F894FA9AF99AAB
S1230B800FBEF999FECF1FBA85EF91E092BD81BD81E080BD0FB6F894FA9AF99A0FBEF99965
S1230BA0FECF1FBA86EF91E092BD81BD84E180BD0FB6F894FA9AF99A0FBEF999FECF1FBAF9
S1230BC087EF91E092BD81BD8AE580BD0FB6F894FA9AF99A0FBEF999FECF1FBA88EF91E08C
S1230BE092BD81BD88EE80BD0FB6F894FA9AF99A0FBEF999FECF1FBA89EF91E092BD81BDBE
S1230C0083E080BD0FB6F894FA9AF99A0FBE2091310130913201F999FECF1FBA8BEF91E0F1
S1230C2092BD81BD20BD0FB6F894FA9AF99A0FBE2091310130913201F999FECF1FBA8CEF77
S1230C4091E092BD81BD30BD0FB6F894FA9AF99A0FBE2091330130913401F999FECF1FBA4D
S1230C608DEF91E092BD81BD20BD0FB6F894FA9AF99A0FBE2091330130913401F999FECF9A
S1230C801FBA8EEF91E092BD81BD30BD0FB6F894FA9AF99A0FBE2091770330917803F999D1
S1230CA0FECF1FBA8FEF91E092BD81BD20BD0FB6F894FA9AF99A0FBE209177033091780385
S1230CC0F999FECF1FBA80E092E092BD81BD30BD0FB6F894FA9AF99A0FBEF999FECF1FBA0F
S1230CE087E092E092BD81BD8CED80BD0FB6F894FA9AF99A0FBEF999FECF1FBA83E092E082
S1230D0092BD81BD86EE80BD0FB6F894FA9AF99A0FBE8CE192E028ECF999FECF1FBA92BDD2
S1230D2081BD20BD0FB6F894FA9AF99A0FBE019632E08C32930781F7F999FECF1FBA8FE827
S1230D4091E092BD81BD82E280BD0FB6F894FA9AF99A0FBEF999FECF1FBA86E092E092BD4C
S1230D6081BD81E080BD0FB6F894FA9AF99A0FBE12BC11BC08958F929F92AF92BF92CF92D1
S1230D80DF92EF92FF920F931F93CF93DF93C0E0D0E035E0832E32E0932E23EDA22E23E0D8
S1230DA0B22EF999FECF92BC81BCF89A60B5F999FECFB2BCA1BCF89AE0B46E01CC0CDD1C2E
S1230DC02FEF31E0C20ED31EF6012081318170E080E090E040E050E00E948E2DFF2400E005
S1230DE010E0A80197010E948E2D24E630E040E050E00E94E02D79018A01C801B70124EFAF
S1230E0031E040E050E00E948E2D28EC30E040E050E0E20EF31E041F151FA80197010E9461
S1230E20E02DCA01B9012FEF30E040E050E00E948E2D25E030E040E050E00E94E02D82E0CB
S1230E40220F331F441F551F8A95D1F7CA01B90124E630E040E050E00E94E02DF601318304
S1230E6020832196C732D10509F09BCFC0E0D0E009EC802E03E0902E13EDA12E13E0B12EAD
S1230E80F999FECF92BC81BCF89A60B5F999FECFB2BCA1BCF89AE0B46E01CC0CDD1C2DE41C
S1230EA032E0C20ED31EF6012081318170E080E090E040E050E00E948E2DFF2400E010E051
S1230EC0A80197010E948E2D24E630E040E050E00E94E02D79018A01C801B70124EF31E0AD
S1230EE040E050E00E948E2D28EC30E040E050E0E20EF31E041F151FA80197010E94E02D85
S1230F00CA01B9012FEF30E040E050E00E948E2D25E030E040E050E00E94E02DA2E0220FA6
S1230F20331F441F551FAA95D1F7CA01B90124E630E040E050E00E94E02DF6013183208391
S1230F402196C732D10509F09BCFC0E0D0E0FAEC8F2EF3E09F2EE3EDAE2EE3E0BE2EF99924
S1230F60FECF92BC81BCF89A60B5F999FECFB2BCA1BCF89AE0B46E01CC0CDD1C2BE932E0B8
S1230F80C20ED31EF6012081318170E080E090E040E050E00E948E2DFF2400E010E0A801D9
S1230FA097010E948E2D24E630E040E050E00E94E02D79018A01C801B70124EF31E040E055
S1230FC050E00E948E2D28EC30E040E050E0E20EF31E041F151FA80197010E94E02DCA01F9
S1230FE0B9012FEF30E040E050E00E948E2D25E030E040E050E00E94E02D62E0220F331F7F
S1231000441F551F6A95D1F7CA01B90124E630E040E050E00E94E02DF6013183208321968B
S1231020C732D10509F09BCFC0E0D0E034E0832E32E0932E23EDA22E23E0B22EF999FECF70
S123104092BC81BCF89A60B5F999FECFB2BCA1BCF89AE0B46E01CC0CDD1C29EE32E0C20ED1
S1231060D31EF6012081318170E080E090E040E050E00E948E2DFF2400E010E0A801970130
S12310800E948E2D24E630E040E050E00E94E02D79018A01C801B70124EF31E040E050E0DC
S12310A00E948E2D28EC30E040E050E0E20EF31E041F151FA80197010E94E02DCA01B9018E
S12310C02FEF30E040E050E00E948E2D25E030E040E050E00E94E02D82E0220F331F441FD5
S12310E0551F8A95D1F7CA01B90124E630E040E050E00E94E02DF601318320832196C732F5
S1231100D10509F09BCFDF91CF911F910F91FF90EF90DF90CF90BF90AF909F908F9008951D
S1231120EAE7F0E0108210927C0080E880BF87EE808311B885E090E09093F9038093F80370
S123114088E790E09093ED038093EC0384E690E09093FB038093FA03909303048093020449
S123116086E490E09093FD038093FC0308950F931F93CF93DF93282F30E0F901EE0FFF1F1B
S1231180EE5FFE4F0081118183E0033F180718F0E2E3F0E04AC083E00F3D180718F0EAE093
S12311A0F0E043C0A0E0B0E087E290E0289FA001299F500D389F500D1124EA01CA0FDB1FBB
S12311C0CC0FDD1FC150DE4F888199818017910730F5FD013197E40FF51FEE0FFF1FE15066
S12311E0FE4F208131816081718148815981FD01EE0FFF1FEE0FFF1FEA0FFB1F3596201B88
S1231200310BC901880F991F880F991F641B750B820F931F0E94B92DE60FF71F06C01196E4
S1231220A732B10551F6E8ECF0E0CF01DF91CF911F910F9108950F931F93CF93DF93AC01CE
S1231240E0E0F0E0EF01CC0FDD1FDE01A95CBC4F8D919C91119748175907C0F56D917C91D2
S12312603197EE0FFF1FDF01A95CBC4F8D919C911197681B790B8D919C91C15BDC4F288162
S12312803981E15BFC4F00811181481B590B84E690E0DC014A9FC0014B9F900D5A9F900DB1
S12312A011240E94B92D201B310B0190F081E02D629FC001639F900D729F900D112464E659
S12312C070E00E94B92D6E0F7F1F09C03196EA30F10509F0B7CF6091630370916403CB016D
S12312E0DF91CF911F910F9108958091EC039091ED03282F205527FF0AC080911401909119
S123130015019C01220F331F280F391F1FC02F312CF0209114013091150118C0409114014E
S123132050911501332727FD309588E290E0821B930B9C01249FC001259F900D349F900D68
S123134011246AE070E00E94B92D9B01C90108950F931F93CF93DF93AC0180917A039091AB
S12313607B034817590718F4E0EFF0E057C080919603909197038417950718F4E0E0F0E032
S12313804DC0E1E0F0E0EF01CC0FDD1FDE01A658BC4F8D919C91119748175907C0F56D9197
S12313A07C913197EE0FFF1FDF01A658BC4F8D919C911197681B790B8D919C91E856FC4F82
S12313C020813181C856DC4F08811981481B590B84E690E0DC014A9FC0014B9F900D5A9FA2
S12313E0900D11240E94B92D201B310B0190F081E02D629FC001639F900D729F900D1124C5
S123140064E670E00E94B92DE61BF70B07C03196EE30F10509F0B7CFEEEFF0E0CF01DF9195
S1231420CF911F910F91089580917204882359F08CED95E09093380180933701109287041E
S1231440109286042AC080917204882349F08CED95E0909338018093370184E690E019C0BF
S123146080917204882349F08CED95E090933801809337018AEF90E00CC080917204882381
S123148061F08CED95E0909338018093370184EF91E09093870480938604F89480915A0438
S12314A090915B048A5A9A4AC1F080915A0490915B048555954589F0789480916D07909161
S12314C06E07806490936E0780936D0784EF91E090933801809337010AC0789480916D07AA
S12314E090916E078F7B90936E0780936D07F89480915C0490915D048F3F89F07894809146
S12315006D0790916E07806890936E0780936D0784EF91E090933801809337010AC0789455
S123152080916D0790916E078F7790936E0780936D078091370190913801892BB1F15E9A76
S123154020918604309187042115310511F45E9A19C08091840490918504029798F48BB11A
S12315608295869586958370809581708295880F880F807C9BB19F7B982B9BB93093850417
S12315802093840480918404909185040197909385048093840480913701909138010197AF
S12315A0909338018093370108955E981092870410928604089580916D0790916E079F77C6
S12315C090936E0780936D07809100019091010197FD44C08091EA0380FF32C020915104A6
S12315E03091520480912101909122018C599F4F8217930720F441E050E060E832C0209103
S1231600510430915204809121019091220149978217930720F441E050E068E022C0209190
S12316205104309152048091210190912201845690408217930790F441E050E064E011C0FC
S1231640209151043091520480912101909122018217930718F440E050E802C040E050E049
S123166060E020916D0730916E07CA019927869597958827822B932B90936E0780936D07C0
S123168020916D0730916E07CA0180709078822B932B90936E0780936D078091000190916B
S12316A0010192FF32C0209151043091520480913101909132018217930738F52091510487
S12316C030915204809133019091340128173907E0F4809127012091F8033091F90390E0EF
S12316E08217930794F080916D0790916E07946090936E0780936D078091EA0380FF03C0C1
S1231700416068600BC0506809C080916D0790916E079B7F90936E0780936D072091FA030E
S12317203091FB0380913A0190E08217930734F480913A01882311F04061686080916B04EE
S12317402091FC033091FD0390E08F5B9F4F8217930774F480916B04882351F04062809112
S1231760510490915204895B9B40A0F0646012C080916B042091FC033091FD0390E0C296FB
S1231780821793073CF480916B04882319F0406271E001C070E080916A04209102043091B3
S12317A0030490E0C296821793076CF480916A04882349F040648091510490915204855CFE
S12317C0994008F06460772321F082E380934D0402C010924D04309906C040FD02C057FF63
S12317E009C0417050785093700440936F046093710406C01092700410926F041092710496
S1231800609372040895809100019091010193FFFCC0339906C0809178048F5F809378049F
S123182002C01092780480917804853108F454C010927304209151043091520480917703B0
S1231840909178038217930778F480916F049091700482609093700480936F0480917104AB
S123186088608093710409C080916F04909170048D7F9093700480936F048091EA0383FF69
S123188016C08091510490915204855C994078F080916F04909170048460909370048093C8
S12318A06F048091710482608093710409C080916F04909170048B7F9093700480936F04B8
S12318C08091740490917504909377048093760484E3809378048EC080917604909177044B
S12318E0892B09F45CC080917604909177040197909377048093760480917304823099F06A
S1231900833030F4882351F0813009F073C019C08330A9F1843009F06DC031C01092770415
S12319201092760467C080916F049091700484609093700480936F048091710482608093CB
S12319407104209151043091520480917703909178038217930768F480916F049091700422
S123196082609093700480936F0480917104806836C080916F04909170048D7F0BC09091EF
S12319808F04809179038917F0F080916F04909170048B7F9093700480936F042BC02091C7
S12319A080043091810421153105E1F080915104909152048D5D9540A8F021503040309344
S12319C081042093800480916F049091700484609093700480936F048091710482608093B2
S12319E0710408C0109283041092820410928104109280048091710481FF07C080913001F9
S1231A0080FF03C084E68093B40408959C018091EA0384FF19C0C901C2979C01B3E0220F33
S1231A20331FBA95E1F7880F991F280F391F2455354F442737FD4095542F60E579E784E04E
S1231A4090E00E94022E20C08091EA0385FD02C024E61AC0C901C2979C01F3E0220F331F24
S1231A60FA95E1F7880F991F280F391F2455354F442737FD4095542F60E579E784E090E0B0
S1231A800E94022E2C592695822F08950F931F93DF93CF93CDB7DEB760970FB6F894DEBFBC
S1231AA00FBECDBFA89582E50E94A52C83E10E94A52C8091510490915204892F0E94A52CD3
S1231AC080915104909152040E94A52C80910204909103040E94A52C80918B0490918C04AF
S1231AE08E5C0E94A52C8091EC039091ED030E94A52C8091FA039091FB030E94A52C809150
S1231B00F8039091F9030E94A52C8091F4039091F5030E94A52C80915804909159046091C6
S1231B20180170E00E94B92D862F0E94A52C809157040E94A52C80915504909156040E9422
S1231B40A52C20916D0730916E078091FA059091FB058870832B0E94A52C80916D07909165
S1231B606E070E94A52C809120060E94A52C80918F070E94A52C8091F2039091F3030E94F6
S1231B80A52C8091FC059091FD05969587950E94A52C86B1869586958695817089831A8260
S1231BA081E090E09C838B8386B1869581708D831E8286B181708F831886809171048987C2
S1231BC01A8680916F04909170049C878B878091F6039091F7039E878D87809171048F8719
S1231BE0188A80918A04E82FF0E0EE0FFF1F8E010F5F1F4FE00FF11F91818295807F892B58
S1231C000E94A52C80918A0490E0880F991F080F191FF80180810E94A52C8DEA0E94A52C49
S1231C2080918A048F5F80938A04883010F010928A0460960FB6F894DEBF0FBECDBFCF91ED
S1231C40DF911F910F9108958F929F92AF92BF92CF92DF92EF92FF920F931F93CF93DF9333
S1231C60A89588E10FB6F89480936000109260000FBE0E94EE2C882311F40C94C2150E94A2
S1231C80822C90938904809388048336910509F471C48436910508F049C08035910509F429
S1231CA013C58135910508F58134910509F4D4C08234910568F48932910509F49FC6843311
S1231CC0910509F449C78832910509F05BC76CC68634910509F427C28D34910509F420C353
S1231CE08534910509F04EC773C18735910509F44EC58835910568F48335910509F4D6C657
S1231D008535910509F4D3C58235910509F03AC781C58136910509F44DC08236910508F0B0
S1231D2026C48835910509F02DC70EC68037910509F4F1C481379105E8F48736910509F428
S1231D409DC48836910548F48536910509F469C38636910508F0A3C110C48D36910509F43C
S1231D609EC28F36910509F406C68936910509F009C75EC4853F910509F4B3C1863F910575
S1231D8068F48937910509F463C68A37910509F44CC48837910509F0F5C647C4873F910593
S1231DA089F1873F910508F41BC2883F910509F0E9C6AFC081E60E94A52C80EA0E94A52C45
S1231DC010928904109288040EC0E35DF94F80810E94A52C809188049091890401969093D3
S1231DE0890480938804E0918804F0918904E03AF10558F38FEF99E50197F1F7000000C011
S1231E008EE927C087EF0E94A52C80EA0E94A52C10928904109288040EC0E353F94F8081F0
S1231E200E94A52C809188049091890401969093890480938804E0918804F0918904E03AD5
S1231E40F10558F38FEF99E50197F1F7000000C088E00E94A52C96C610928904109288046D
S1231E6000E010E0BFEFEB2EB3EBFB2E0E94EE2C882309F446C0C0918804D0918904C03AD1
S1231E80D10579F50E94822C90938904809388048E3B910579F481E40E94A52C81E00E94B4
S1231EA0A52C81E00E94A52C8EEB0E94A52C06E11AEF27C081E40E94A52C81E00E94A52C0A
S1231EC080E00E94A52C8EEB0E94A52CC7010197F1F7000000C0E0917E04F0917F040995A2
S1231EE010C00E94822CC35DD94F888380918804909189040196909389048093880400E05A
S1231F0010E00F5F1F4F8AEF0030180708F4AECF39C61092890410928804C0E0D0E0AFEF66
S1231F20EA2EA3EBFA2E0E94EE2C882309F449C00091880410918904003A110579F50E94B7
S1231F40822C90938904809388048730910579F488EF0E94A52C81E00E94A52C81E00E9405
S1231F60A52C87E00E94A52CC6E1DAEF2AC088EF0E94A52C81E00E94A52C80E00E94A52CC7
S1231F8087E00E94A52CC7010197F1F7000000C0E0917E04F0917F04099513C000561F4F2F
S1231FA00E94822C035D194FF8018083809188049091890401969093890480938804C0E038
S1231FC0D0E02196FAEFC030DF0708F4ACCFDAC5C0E0D0E0F8E1FF2E0AEF10E00E94EE2CC6
S1231FE0882309F455C00E94822C8A3B910509F0C9C50FB6F894F0926000109260000FBEEC
S123200010928904109288043BC0885B0E94A52C8DEF0E94A52C8091880490918904809FB5
S1232020E001819FD00D909FD00D112409C0F999FECFD2BDC1BDF89A80B50E94A52C219657
S123204020918804309189042F5F3F4F209FC001219F900D309F900D112421503040C81797
S1232060D90728F3822F885B80950E94A52C80918804909189040196909389048093880414
S123208080918804909189048430910508F4BDCF21968AEFC030D80708F4A0CF73C586E611
S12320A00E94A52C80EA0E94A52C10928904109288040EC0E654FB4F80810E94A52C809198
S12320C088049091890401969093890480938804E0918804F0918904E03AF10558F389E904
S12320E0B8CE85EF0E94A52C80EA0E94A52C10928904109288040EC0E65AFA4F80810E943B
S1232100A52C809188049091890401969093890480938804E0918804F0918904E03AF1059E
S123212058F38AE096CE109289041092880400E010E0EFEFEE2EE3EBFE2E0E94EE2C8823FA
S123214009F446C0C0918804D0918904C03AD10579F50E94822C9093890480938804893B0C
S1232160910579F486E40E94A52C81E00E94A52C81E00E94A52C89EB0E94A52C06E11AEFFC
S123218027C086E40E94A52C81E00E94A52C80E00E94A52C89EB0E94A52CC7010197F1F7A1
S12321A0000000C0E0917E04F0917F04099510C00E94822CC654DB4F888380918804909199
S12321C089040196909389048093880400E010E00F5F1F4FEAEF00301E0708F4AECFD2C49F
S12321E01092890410928804C0E0D0E07FEFE72E73EBF72E0E94EE2C882309F449C000912A
S1232200880410918904003A110579F50E94822C90938904809388048930910579F486EF72
S12322200E94A52C81E00E94A52C81E00E94A52C89E00E94A52CC6E1DAEF2AC086EF0E9432
S1232240A52C81E00E94A52C80E00E94A52C89E00E94A52CC7010197F1F7000000C0E091AD
S12322607E04F0917F04099513C000561F4F0E94822C06541B4FF8018083809188049091D1
S1232280890401969093890480938804C0E0D0E02196FAEFC030DF0708F4ACCF73C48DE6E0
S12322A00E94A52C89E00E94A52C80911F01909120010E94A52C80911F0190912001892FBA
S12322C00E94A52C80912501909126010E94A52C8091250190912601892F0E94A52C8091DA
S12322E00001909101010E94A52C8091000190910101892F0E94A52C809113010E94A52C4B
S1232300809112010E94A52CF999FECF8AE090E092BD81BDF89A80B50E94A52C82E999CD51
S12323201092890410928804AA24BB246AE0862E912C0E94EE2C8A3008F469C00E94822CE9
S12323409093200180931F0100911F01109120010E94822CD82ECC240C0D1D1D1093200132
S123236000931F010E94822C909326018093250100912501109126010E94822CF82EEE24CC
S12323800E0D1F1D10932601009325010E94822C90930101809300010091000110910101A1
S12323A00E94822CD82FC0E00C0F1D1F10930101009300010E94822C809313010E94822CCB
S12323C0809312010E94822CF999FECF1FBA92BC81BC80BD0FB6F894FA9AF99A0FBE0E949C
S12323E0C9260E94822C823B910561F40E94BC04E0917E04F0917F0409955FE6A52E5AEF9A
S1232400B52E05C0E0917E04F0917F0409950894A11CB11C80E0A8168AEFB80608F489CFAC
S1232420B1C385E60E94A52C83E10E94A52C10928904109288040EC0EB51FE4F80810E9418
S1232440A52C809188049091890401969093890480938804E0918804F0918904EA30F1055B
S123246058F38091190190911A016091180170E00E94B92D862F0E94A52C80911C0190914D
S12324801D016091180170E00E94B92D862F0E94A52C8FEF95E30197F1F7000000C08091C9
S12324A02A010E94A52C80912B010E94A52C80912C010E94A52C80912D010E94A52C809156
S12324C014019091150166E070E00E94B92D862F0E94A52C809127010E94A52CF999FECF5B
S12324E08EE691E092BD81BDF89A80B50E94A52C8AE90E94A52C8CE60E94A52C84E10E945A
S1232500A52C10928904109288040EC0E050FA4F80810E94A52C80918804909189040196EC
S12325209093890480938804E0918804F0918904EA30F10558F310928904109288040EC0B7
S1232540E050FA4F80890E94A52C809188049091890401969093890480938804E091880454
S1232560F0918904EA30F10558F383E972CC0E94A40008C30E94D90005C381E50E94A52C17
S123258080E10E94A52C8091B8039091B9030E94A52C80919E0790919F070E94A52C809146
S12325A0A0079091A1070E94A52C8091A2079091A3070E94A52C8091A4079091A5070E9411
S12325C0A52C8091A6079091A7070E94A52C8091A8079091A9070E94A52C8091F4039091F9
S12325E0F5030E94A52C809171040E94A52C80916F04909170040E94A52C8091B407809506
S12326000E94A52C80918F040E94A52C809120060E94A52C84E00E94A52C85E00E94A52CD3
S123262086E00E94A52C8EEA14CC0E94460DAAC20E94EE2C8530E0F30E94822CC82FD0E0C9
S12326400E94822CC817D90709F09CC20E94822C8C0190938904809388040E94822C081775
S1232660190709F08FC20E94822C8639910509F089C280918804C35DD94F4BC00E94EE2C57
S12326808530E0F30E94822CC82FD0E00E94822CC817D90709F076C20E94822C8C01909377
S12326A08904809388040E94822C0817190709F069C20E94822C8839910509F063C2809161
S12326C08804C654DB4F25C00E94EE2C8530E0F30E94822CC82FD0E00E94822CC817D907F7
S12326E009F050C20E94822C8C0190938904809388040E94822C0817190709F043C20E9470
S1232700822C8F3A910509F03DC280918804CB5BDE4F888337C2C0E0D0E00E94EE2C8230FE
S123272080F10E94822C0E94822C8F38910509F029C210928904109288041CC0EB5BFE4F77
S1232740108180E70E94A52C82E00E94A52C809188040E94A52C812F0E94A52C8FE80E94E9
S1232760A52C809188049091890401969093890480938804E0918804F0918904E03AF10538
S1232780E8F22196EAEFC030DE0739F6FBC10E94EE2C8530E0F30E94822CE82ED92E0E94B8
S12327A0822CF82E0E94822C8C0190938904809388040E94822C0817190709F0E3C18E2D2E
S12327C09D2DDF2DC0E08E01080F191F0E94822C883A9105C9F4C80161E670E00E94632DAA
S12327E0BC0160708091880490918904682B792B7093890460938804C80149E650E00E94ED
S1232800792D12BC11BCBEC1E0917E04F0917F040995BDCFAA24BB240E94EE2C833008F4BB
S12328203CC00E94822C082F992E0E94822C182F0E94822C8D3A910509F0A4C1F999FECF49
S1232840802F992DD12ECC24E601C80FD91FD2BDC1BDF89A90B5F999FECF2196D2BDC1BD53
S12328602197F89A80B5F82EEE248701090F111D84E50E94A52C84E00E94A52C802F0E94CB
S1232880A52C8C2F0E94A52C8D2F0E94A52C812F0E94A52C8BEA0E94A52C0894A11CB11CD5
S12328A0F0E0AF16FAEFBF0609F0B6CF6BC1AA24BB240E94EE2C833008F43CC00E94822CC3
S12328C0082F992E0E94822C182F0E94822C8A3A910509F057C1F999FECF802F992DD12ED1
S12328E0CC24E601C80FD91FD2BDC1BDF89A90B5F999FECF2196D2BDC1BD2197F89A80B5A8
S1232900F82EEE248701090F111D85E50E94A52C84E00E94A52C802F0E94A52C812F0E9485
S1232920A52C8C2F0E94A52C8D2F0E94A52C8AEA0E94A52C0894A11CB11C80E0A8168AEFC1
S1232940B80609F0B6CF1EC1C0E0D0E00E94EE2C882359F00E94822C873A910509F012C1E5
S1232960E0917E04F0917F0409952196EAEFC030DE0761F707C1C0E0D0E00E94EE2C882382
S123298069F00E94822C8039910509F0FBC00E940B01E0917E04F0917F0409952196FAEFA4
S12329A0C030DF0751F7EEC0C0E0D0E00DE611E00E94EE2C8823E1F00E94822C873D910531
S12329C009F0E0C08091F8039091F903F999FECF1FBA12BD01BD80BD0FB6F894FA9AF99AB7
S12329E00FBE12BC11BCE0917E04F0917F04099521968AEFC030D807D9F6C4C0C0E0D0E034
S1232A000EE611E00E94EE2C8823E1F00E94822C863D910509F0B6C08091F8039091F90354
S1232A20F999FECF1FBA12BD01BD80BD0FB6F894FA9AF99A0FBE12BC11BCE0917E04F0913C
S1232A407F0409952196EAEFC030DE07D9F69AC0C0E0D0E00E94EE2C823010F10E94822CB4
S1232A60892B09F08FC00E94822C86389105C1F489E70E94A52C85E00E94A52C8FEC0E9425
S1232A80A52C8FE30E94A52C88E00E94A52C82EA0E94A52C85ED0E94A52C86E80E94A52CFC
S1232AA02196FAEFC030DF07A9F66CC0C0E0D0E00E94EE2C823008F448C00E94822C892B0B
S1232AC009F043C00E94822C8C3A910509F05AC083E50E94A52C88E00E94A52C80915A0412
S1232AE090915B040E94A52C80915A0490915B04892F0E94A52C80912B0690912C060E948E
S1232B00A52C80912B0690912C06892F0E94A52C80912406909125060E94A52C80912406EB
S1232B2090912506892F0E94A52C8091BA079091BB070E94A52C8091BA079091BB07892F85
S1232B400E94A52C8CEA0E94A52C21968AEFC030D80709F0ADCF16C0C0E0D0E00E94EE2CBF
S1232B60823058F00E94822C892B61F40E94822C8B3C910511F40E9426012196EAEFC03003
S1232B80DE0761F7A895DF91CF911F910F91FF90EF90DF90CF90BF90AF909F908F90089542
S1232BA02F923F924F925F926F927F928F929F92AF92BF92CF92DF92EF92FF920F931F937F
S1232BC0CF93DF9310926E0710926D070E94F02B259A249A00002D9A2C9A81E080932A0685
S1232BE0569A8093FE05209A219A219A209A289A299A299A289A549A559A5C9A5D9A229A51
S1232C00239A569A2A9A2B985E9800000000529853983B98439A3A98429A3998419A3898D7
S1232C20409A0E94F72BF999FECF8AE591E092BD81BDF89A80B5809360040E94AB1C0E94DD
S1232C40C9260E94E02B10927A0010927C0080E880BF87EE80937A0011B885E090E0909330
S1232C60F9038093F80388E790E09093ED038093EC0384E690E09093FB038093FA03909324
S1232C8003048093020486E490E09093FD038093FC030E94BB062A9A2B98F999FECF87E051
S1232CA090E092BD81BDF89A80B512BC11BC85FFEEC080910001909101019F7D9093010109
S1232CC0809300010E94BC040E9443050E94D9000E94A4000E940B01F999FECF1FBA8AE07F
S1232CE090E092BD81BD86E080BD0FB6F894FA9AF99A0FBEF999FECF1FBA8BE090E092BD89
S1232D0081BD89E180BD0FB6F894FA9AF99A0FBEF999FECF1FBA8CE090E092BD81BD8EE175
S1232D2080BD0FB6F894FA9AF99A0FBEF999FECF1FBA8EE090E092BD81BD8EE180BD0FB6F9
S1232D40F894FA9AF99A0FBE80E090E0FC01EB51FE4FE081F999FECF1FBA825A9E4F92BDE8
S1232D6081BDE0BD0FB6F894FA9AF99A0FBE8D5591408A30910551F780E090E0FC01E65DD4
S1232D80FE4FE081F999FECF1FBA87599E4F92BD81BDE0BD0FB6F894FA9AF99A0FBE88562F
S1232DA091408430910551F780E090E0FC01E050FA4FE081F999FECF1FBA8E589E4F92BDAB
S1232DC081BDE0BD0FB6F894FA9AF99A0FBE815791408A30910551F780E090E0FC01E05091
S1232DE0FA4F2089F999FECF1FBA84589E4F92BD81BD20BD0FB6F894FA9AF99A0FBE8B574B
S1232E0091408A30910551F720912306F999FECF1FBA81E791E092BD81BD20BD0FB6F8949F
S1232E20FA9AF99A0FBE2091140130911501F999FECF1FBA8DE090E092BD81BDC90166E04B
S1232E4070E00E94B92D60BD0FB6F894FA9AF99A0FBEF999FECF1FBA8DE691E092BD81BD8B
S1232E6084E180BD0FB6F894FA9AF99A0FBEF999FECF1FBA8EE691E092BD81BD81EE80BD11
S1232E800FB6F894FA9AF99A0FBE12BC11BC0E94F3000E94260120E030E0F999FECF205F02
S1232EA03F4F32BD21BD20513040F89A80B5F901E654FB4F80832F5F3F4F81E0203438077A
S1232EC061F712BC11BC0E947600809100019091010185FD07C080916F008B7F80936F0059
S1232EE02D9A2C9A80912901882311F480E801C080E480933B011092EB03809114019091A3
S1232F0015018D5A9D4030F08CEA9DE0909315018093140110924E0486B3866086BB7894FF
S1232F208AEA0E94A52C80E00E94A52C85E50E94A52C86B1869581708093620480916E00BB
S1232F40836080936E002A9AFF24F394F4E02F2EE7E8BE2E77E0A72E63E4962E56E4852E8B
S1232F604BE4C42ED12C33E0732E24E4622E94E6E92E82E0582E05E4402E11E4312E2B9AFA
S1232F80A89580915104909152048635910568F180914E04882349F580916D0790916E0702
S1232FA09F7E90936E0780936D0780916F00856080936F0080916E00836080936E002A9A43
S1232FC0F0924E0480916D0790916E07806290936E0780936D0780916D0790916E079062F0
S1232FE090936E0780936D074AC020914E04213009F045C080915104909152048234910529
S123300008F03DC080916F008D7F80936F00809170008C7F8093700080916F008B7F8093FD
S12330206F0080916E00836080936E0080916D0790916E078F7D90936E0780936D078091E3
S12330406D0790916E07877F90936E0780936D07289A299A299A289A5C9A5D9A2D9A2C9AB9
S123306020932A0610924E0480916D0790916E079F7D90936E0780936D0710924C0480911C
S12330804E048130D9F480916F00826080936F008091700083608093700080916E0083602F
S12330A080936E0080916D0790916E07886090936E0780936D072A9A2B9A15C010924C0419
S12330C02D9A2C9AF0922A0610924C041092B30010925904109258048091430190914401AE
S12330E0892B09F42A988091EB03833009F4CAC0843018F4882371F071C0853009F4E8C1C8
S1233100853008F422C1863009F499C1873009F068C221C280914F04909150048536910523
S123312008F461C2E091EB03F0E080917800909179008C7F65E070E00E94B92DEE0FFF1FD7
S1233140E45DFB4F718360838091EB03C82FD0E0E091EB03F0E0EE0FFF1FE451FC4F808198
S12331609181E091EB03F0E0EE0FFF1FE45DFB4F20813181880F991F880F991F820F931F30
S1233180880F991F6AE070E00E94B92DCC0FDD1FC451DC4F798368831092500410924F04D1
S12331A0F092EB0330927C000E94240E0E9475099093170180931601809143019091440149
S12331C0892B51F08091430190914401019790934401809343012A9AA89505C280914F04B8
S12331E0909150048536910508F4FDC11092500410924F04A8958091EB03813031F580913C
S12332000801909109012091780030917900820F931F96958795909309018093080183E0DD
S12332200E94B7089093EF038093EE038091EE039091EF039093030480930204E0929307AC
S12332405092EB0340927C00CEC180910201909103012091780030917900820F931F9695B3
S123326087959093030180930201D092F103C092F003D092FD03C092FC037092EB036092C1
S12332807C00B1C180914F04909150048536910508F4A9C1E091EB03F0E0809178009091D3
S12332A079009695879596958795EE0FFF1FE45DFB4F918380838091EB03C82FD0E0E0912F
S12332C0EB03F0E0EE0FFF1FE451FC4F80819181E091EB03F0E0EE0FFF1FE45DFB4F208108
S12332E03181880F991F880F991F820F931F880F991F6AE070E00E94B92DCB01CC0FDD1F23
S1233300C451DC4F998388831092500410924F042092EB0380913B0180937C000E94240E07
S1233320A89580916E048F5F80936E04843010F010926E0480916E04982F91709093AF046D
S123334086958170809326064EC180914F04909150048159914008F446C1809129018823A2
S123336029F1E091EB03F0E080917800909179009695879596958795EE0FFF1FE45DFB4FA9
S123338091838083A091EB03B0E0E091EB03F0E0EE0FFF1FE45DFB4F80819181AA0FBB1FE8
S12333A0A451BC4F11969C938E933EC0E091EB03F0E08091780090917900EE0FFF1FE45D66
S12333C0FB4F918380838091EB03C82FD0E0E091EB03F0E0EE0FFF1FE451FC4F0081118105
S12333E0E091EB03F0E0EE0FFF1FE45DFB4F808191810E94A8099C01220F331F280F391FDF
S1233400C801F3E0880F991FFA95E1F7801B910B820F931F6AE070E00E94B92DCC0FDD1FE3
S1233420C451DC4F798368831092500410924F0485E08093EB03B0927C00A895D4C0809170
S12334404F04909150048536910508F4CCC0E091EB03F0E08091780090917900969587952E
S123346096958795EE0FFF1FE45DFB4F91838083A091EB03B0E0E091EB03F0E0EE0FFF1F4B
S1233480E451FC4F20813181E091EB03F0E0EE0FFF1FE45DFB4F80819181820F931F880F93
S12334A0991F9695879596958795AA0FBB1FA451BC4F11969C938E931092500410924F044D
S12334C0A092EB0390927C000E94240EA8958BC080914F0490915004893C910508F483C05B
S12334E0E091EB03F0E08091780090917900EE0FFF1FE45DFB4F91838083A091EB03B0E00A
S1233500E091EB03F0E0EE0FFF1FE451FC4F20813181E091EB03F0E0EE0FFF1FE45DFB4FB5
S123352080819181820F931F96958795AA0FBB1FA451BC4F11969C938E93109250041092C8
S12335404F0426E02093EB0382E480937C000E94240EA89548C080914F04909150048536CB
S1233560910508F440C0E091EB03F0E08091780090917900969587959695879590E0EE0F68
S1233580FF1FE45DFB4F91838083A091EB03B0E0E091EB03F0E0EE0FFF1FE451FC4F20814D
S12335A03181E091EB03F0E0EE0FFF1FE45DFB4F80819181820F931F96958795AA0FBB1F50
S12335C0A451BC4F11969C938E931092500410924F041092EB0380927C000E94240EA895D6
S12335E002C0F092EB0380914F049091500401969093500480934F0480915104909152046B
S12336008F55914008F448C08091C00787FF02C0E0E002C0E091C007809191078F5F809369
S1233620910790919107809192079817B8F1109291072091FA033091FB03AE2FB0E0FD0121
S1233640E159F84F808190E02817390754F480918F07843634F480918F0790919007890F2D
S123366012C02091FA033091FB03A159B84F8C9190E0281739074CF080918F0782302CF049
S123368080918F07815080938F0780918F0785362CF0E0928F0702C0F0928F07809151043F
S12336A0909152048739910508F46DC0809127012091F8033091F90390E0489682179307ED
S12336C00CF461C08091B6049091B70401969093B7048093B6042091B6043091B7048091E4
S12336E0B8049091B9042817390708F440C01092B7041092B60420915104309152048091CA
S1233700B0049091B1040A972817390730F49091B4048091B504890F15C020915104309100
S123372052048091B0049091B10449968217930758F49091B4048091B304891728F48091C8
S1233740B40481508093B4049091B4048091B204891718F48091B20408C09091B40480914C
S1233760B304981720F48091B3048093B40480915104909152048A58924038F48091B204B4
S12337808093B40402C01092B4048091EA0382FF4EC08091510490915204855F914008F423
S12337A046C08091510490915204805D974008F03EC0809127012091F8033091F90390E066
S12337C00496821793079CF12091F8033091F9038091650490E001968217930744F1809128
S12337E0660490916704A0916804B09169040196A11DB11D8093660490936704A0936804B7
S1233800B09369048091660490916704A0916804B091690481549D40A340B04008F1F092A2
S1233820640480916D0790916E07916015C08091F8039091F90380936504109266041092E8
S1233840670410926804109269041092640480916D0790916E079E7F90936E0780936D077B
S12338600E94DB0A0E94030C0E94140A809100019091010180FF67C08091300180FF11C0DF
S12338808091AD04883C28F08091B4048823C9F016C09091B4048091AD048695891790F0AD
S12338A010C08091300182FF0DC08091AD04883C48F080916D0790916E0796FF02C05C9A7E
S12338C001C05C988091300184FF16C08091AD04883C28F080918F0718165CF12CC0209137
S12338E08F078091AD04332727FD3095869590E0821793070CF11FC08091300186FF1CC0EC
S12339008091AD04883CC0F0209151043091520480913501909136018217930760F4209179
S1233920FA033091FB038091610490E08217930714F45D9A01C05D988091AD04883C28F05B
S12339401092AD0402C05C9A5D9A8091AD048F5F8093AD0414CB1092800081EF9FEF9093CB
S123396089008093880085EF9FEF90938B0080938A0080E88093810080EC9AED909385003B
S12339808093840083E090E09093CF038093CE038091CE039091CF038068809381001092ED
S12339A052041092510480916F00876080936F0052985398259A249A2D9A2C9A81E080937A
S12339C02A06F999FECF82E092E092BD81BDF89A80B58093BA03F999FECF81E092E092BDDB
S12339E081BDF89A80B58093BB038091BB038E3039F08091BB03873119F087E18093BB036E
S1233A008091690084608093690080916900816080936900E89A08951F920F920FB60F921A
S1233A2011248F939F938091C1078F5F8093C1078091C107882309F449C080916D07909127
S1233A406E07906190936E0780936D0710924E0480916D0790916E079F7D90936E07809307
S1233A606D0780916F008B7F80936F0080916F008D7F80936F00809170008C7F80937000A5
S1233A8080916E00836080936E002D9A2C9A81E080932A0680916D0790916E078F7D9093C4
S1233AA06E0780936D0780916D0790916E07877F90936E0780936D07289A299A299A289ABC
S1233AC05C9A5D9A109252041092510410928C0410928B0478949F918F910F900FBE0F903C
S1233AE01F9018952091BE073091BF078091BE079091BF07E0918400F09185006AE070E017
S1233B000E94B92D260F371F2E173F07A8F580919A078430E9F480915C0490915D04880F99
S1233B20991F90935D0480935C0480915C0490915D04816090935D0480935C0480918B0467
S1233B4090918C04019690938C0480938B0404C010925D0410925C0481E080939A078091D5
S1233B60B6039091B7039093B9038093B8031092B7031092B60315C080919A078F5F8093C1
S1233B809A0780919A07853061F481E080939A0780918B0490918C04019790938C04809300
S1233BA08B0480918B0490918C048536910530F084E690E090938C0480938B0480918400EC
S1233BC0909185009093BF078093BE0708951F920F920FB60F9211248F939F938091B603D2
S1233BE09091B70301969093B7038093B6039F918F910F900FBE0F901F9018958091A50435
S1233C00882309F466C08091A504813051F42D9A8091B6039091B7039093CA078093C907DF
S1233C200DC08091A504823049F42C9A8091B6039091B7039093B3078093B2078091A6043B
S1233C40882319F41092A5042FC08091A604813099F480918A0090918B004E9690938B009C
S1233C6080938A008091A5048C598093A5048091A5048093A60418C08091A604853619F476
S1233C8085B190E206C08091A604863669F485B190E1892785B980918A0090918B004E961E
S1233CA090938B0080938A008091240690912506892B09F449C08091BC07882309F444C0F4
S1233CC0809124069091250690938B0080938A0008958091BC078823B9F18091BC078130C3
S1233CE091F42091BC0780916D0790916E0793FD08C0213019F0223021F402C02D9801C04B
S1233D002C9881E015C08091BC07823099F42091BC0780916D0790916E0793FD08C021305A
S1233D2019F0223021F402C02D9801C02C9882E08093A5048091BA079091BB0790938B0082
S1233D4080938A001092BC0708951F920F920FB60F9211242F933F934F935F936F937F9357
S1233D608F939F93AF93BF93EF93FF930E94FE1D2A9A7894FF91EF91BF91AF919F918F91C6
S1233D807F916F915F914F913F912F910F900FBE0F901F901895282F80916D0790916E07D6
S1233DA093FD08C0213019F0223021F402C02D9808952C9808951F920F920FB60F92112474
S1233DC08F939F93F89480919B07882309F486C080916F049091700497FD80C0809113014C
S1233DE080958093B4078091B407909120068C59891B8093B4079091FF05943029F19530AA
S1233E0040F4923051F19330B8F4913009F058C009C09731C1F1933609F441C09E3009F054
S1233E204FC023C08091B4078093B20084E08093B100289883E050C08091B40786BD83E02E
S1233E4085BD299884E048C08091B4078093B2009093B100289882E03FC08091B40786BD5A
S1233E6083E085BD299881E037C081E08093D3038091B4078093B20084E08093B1002898BD
S1233E80289887E129C081E08093D4038091B40786BD83E085BD299829988EE01DC081E0E0
S1233EA08093D3038091B4078093B20084E08093B10028982898299829989093FF050EC065
S1233EC08091B4078093B20084E08093B100289828982998299883E68093FF0578949F9167
S1233EE08F910F900FBE0F901F901895EF92FF920F931F93CF93DF93EC0180915F04E7E0D5
S1233F00F0E0E81BF109EE0FFF1FE451FC4F8081918120915E04821B482F50E080912E018B
S1233F2026E0829FC00111249C01249FC001259F900D349F900D112464E670E00E94B92D17
S1233F40CB01603A710508F08FE98093BD078091BD076AE00E94AD2D809396078091960741
S1233F6080311CF08FE0809396078091510490915204885E934008F0AAC0109294078FEFAE
S1233F808093C0078091960724E18202C00111249093560480935504809151049091520450
S1233FA064E670E00E94B92D65506093B9078091510490915204845F914060F41092B9072C
S1233FC0E091B907FF27E7FDF095E25CFE4F808190E0A9C08091B9078430E1F5E091550493
S1233FE0F0915604E35DF94F2081E091B907FF27E7FDF095E25CFE4F6081E091B907FF2736
S1234000E7FDF095E25CFE4F808190E09093FD058093FC05E091FC05F091FD0580915104A3
S1234020909152044091B90730E0220F331F261B3109845F91406CE94602A0011124840FAC
S1234040951FDC012A9FC0012B9F900D3A9F900D11243AC0E091B907FF27E7FDF095E15C38
S1234060FE4F6081E091B907FF27E7FDF095E25CFE4F4081E091B907FF27E7FDF095E25C04
S1234080FE4F808190E09093FD058093FC05E091FC05F091FD0580915104909152042091A2
S12340A0B90770E0641B7109845F91404CE9240290011124820F931F9C01629FC001639F7A
S12340C0900D729F900D112464E670E0D1C08091510490915204875F924250F187EC8093D3
S12340E09407809194076AE00E94AD2D8093C007809196072091C00744E18402C00111240E
S1234100332727FD3095820F931F9093560480935504E0915504F0915604E35DF94F8081FE
S123412090E0880F991F9093FD058093FC05A8C08091510490915204885E934062E370E0F0
S12341400E94B92D60939407809194076AE00E94AD2D8093C007809196072091C00744E1AE
S12341608402C0011124332727FD3095820F931F9093560480935504E0915504F0915604AB
S1234180E35DF94F808190E0880F991F9093FD058093FC058091C00787FD37C08091C0076F
S12341A083319CF5E0915504F0915604E25DF94F4081E0915504F0915604E35DF94F6081BB
S12341C0E091FC05F091FD05309194078091C00726EF8202C0011124830F911D880F991F94
S12341E050E0461B5109DC01A49FC001A59F900DB49F900D11246AE070E00E94CD2DE60FBE
S1234200F71FF093FD05E093FC058091960787FD37C0809196078F309CF5E0915504F09119
S12342205604EF5BF94F4081E0915504F0915604E35DF94F6081E091FC05F091FD05309109
S1234240BD078091960726EF8202C0011124830F911D880F991F50E0461B51099C01249F7F
S1234260C001259F900D349F900D11246AE070E00E94CD2DE60FF71FF093FD05E093FC0539
S123428080916D0790916E07977F90936E0780936D078091FA059091FB05877F9093FB0570
S12342A08093FA0580917104882309F458C08091710487FD27C080917104883088F08091EA
S12342C0990790E083709070892B09F448C08091990767E00E94AD2D992309F440C012C01F
S12342E0809171048430C0F08091990790E083709070892B39F08091990767E00E94AD2D6B
S1234300992369F580916D0790916E07986090936E0780936D0723C080917104823050F0F2
S12343208091FA059091FB0588609093FB058093FA0515C080917104882389F08091FC059A
S12343409091FD058739910550F08091FC059091FD058C5890409093FD058093FC0580916D
S123436099078F5F8093990740918F04445645310CF044E12091FC053091FD0580911201CA
S123438090914D04285B3F4F280F311D291B3109842F4C3E0CF48CEE992787FD9095280F3C
S12343A0391F30938E0420938D0440918D0450918E048091AE042AE08202C0011124840F59
S12343C0951F90938E0480938D0480918D0490918E048D5B92403CF04CEBE42E42E0F42E04
S12343E0012D112D15C080918D0490918E04059734F435E0E32EF12C012D112D09C08091D6
S12344008D0490918E047C010027F7FC0095102F82EC91E0A0E0B0E0E80EF91E0A1F1B1F8A
S123442020915304309154042C0F3D1F40E050E0C801B7010E948E2D28E037E040E050E023
S12344400E94E02DDE01A21BB30BCD01DF91CF911F910F91FF90EF9008950F931F93CF9300
S1234460DF938091CC039091CD039093C8078093C7078091CC039091CD03499708F467C24C
S12344808091C107882349F088EE9DEF9093D1038093D0031092C10753C080915104909178
S12344A052044091D0035091D103895B9B40C0F0E0915304F09154042091CC033091CD0328
S12344C08091BA0390E0241B350BAC01429FC001439F900D529F900D112464E170E017C01E
S12344E0E0915304F09154042091CC033091CD038091BA0390E0241B350BAC01429FC001FA
S1234500439F900D529F900D11246EE170E00E94CD2DCB018E0F9F1F62E070E00E94CD2DC5
S1234520709354046093530410925404109253048091CC039091CD039093D1038093D00331
S123454080914C04893628F480914C048F5F80934C048091510490915204805D974040F4A4
S12345602D9B02C02C9904C02D9A2C9A1092A5048091510490915204C091D003D091D10316
S1234580D0932C06C0932B0620912B0630912C060091CE031091CF0340E050E060E070E470
S12345A089E191E00E94022ECA01B9012EE130E040E050E00E948E2D20EC30E0A901049F90
S12345C09001059F300D149F300D11242050324040E050E00E94E02D30935204209351043E
S12345E020919C0430919D0440919A0450919B04C901880F991F820F931F840F951F969547
S123460087959695879590939D0480939C04809198049091990490939B0480939A048091CD
S12346209604909197049093990480939804809194049091950490939704809396048091D2
S12346409204909193049093950480939404809190049091910490939304809392048091D2
S1234660510490915204909391048093900480915104909152048D5D9540B8F080918F0423
S1234680409190045091910420919C0430919D0490E0821B930B840F951F96958795969524
S12346A08795855B80938F040FC084E680938F04809153049091540464E070E00E94CD2D64
S12346C070935404609353041092C10780915104909152048C529140A0F58091CE039091A3
S12346E0CF03039771F580919A07813051F584E090E09093CF038093CE038091CE0390918B
S1234700CF038068809381008091840090918500969587959695879590938500809384003F
S1234720D695C795D695C795D093D103C093D00380912B0690912C06969587959695879567
S12347403AC080915104909152048F5E9240B8F18091CE039091CF03049789F580919A0776
S1234760813069F583E090E09093CF038093CE038091CE039091CF03806880938100809118
S1234780840090918500880F991F880F991F9093850080938400CC0FDD1FCC0FDD1FD093FD
S12347A0D103C093D00380912B0690912C06880F991F880F991F90932C0680932B0680911E
S12347C02B0690912C060E94761F9093BB078093BA078091FA059091FB0583FF3AC0E09143
S12347E0A704F091A804CF0183709070892B99F420912B0630912C0680912B0690912C066F
S12348006AE070E00E94B92D261B370B3093BB072093BA0718C020913C0180912B069091CD
S12348202C0668E270E00E94B92D30E0629FC001639F900D729F900D11248C599F4F9093D6
S1234840BB078093BA073196F093A804E093A70404C01092A8041092A704809151049091C4
S123486052048A58924038F08091EC039091ED038E3691053CF48CE291E09093C507809386
S1234880C40704C01092C5071092C4078091BA079091BB0720911601309117014091C407B8
S12348A05091C507821B930B841B950B9093B1078093B0078091B0079091B10797FF20C011
S12348C08091B0079091B10720912B0630912C064091BA075091BB07820F931F84179507AF
S12348E078F48091BA079091BB0720912B0630912C064496821B930B9093B1078093B00704
S1234900F89480919A07833011F48EE005C080919A078230E1F487E18093FF0560912B0690
S123492070912C0680E090E028E532E040E050E00E948E2D28E037E040E050E00E94E02D86
S1234940309389002093880081E080939B077894DF91CF911F910F9108951F920F920FB6D6
S12349600F9211242F933F934F935F936F937F938F939F93AF93BF93EF93FF93F89489B11F
S12349808695869581702091600490E030E082179307D9F078940E942D220E94721D80911C
S12349A05A0490915B04880F991F90935B0480935A0480915A0490915B04816090935B0481
S12349C080935A041092FE05BFC120918400309185008091CC039091CD039695879528176B
S12349E0390778F48091510490915204815D974040F081E090E090935B0480935A04789475
S1234A00A3C18091FA059091FB0583FF97C080918400909185009093CD038093CC03109272
S1234A20850010928400789480915A0490915B04880F991F90935B0480935A0481E0809316
S1234A40FE0520913C0180912B0690912C0668E270E00E94B92D30E0629FC001639F900D39
S1234A60729F900D11248C599F4F9093BB078093BA0780915104909152048051974208F044
S1234A8049C080916D0790916E0793FD43C08091BA079091BB0790938B0080938A002091AA
S1234AA02B0630912C0680912B0690912C069695879596958795281B390B30932506209383
S1234AC0240680919A07813021F080919A07833031F42C9882E08093A50481E00DC0809189
S1234AE09A07843021F080919A07823039F42D9881E08093A50482E08093BC078EEB90E0B8
S1234B00909328068093270680916D0790916E079F770FC080912B0690912C068C509E4FA2
S1234B2090938B0080938A0080916D0790916E07906890936E0780936D0706C18091840098
S1234B40909185009093CD038093CC031092850010928400789480915A0490915B04880FF7
S1234B60991F90935B0480935A0481E08093FE0580915104909152048051974208F0DAC0F6
S1234B808091B0079091B107853691050CF44EC01092A5048091510490915204885592403A
S1234BA050F48091BA079091BB07969587959093B1078093B00780915104909152048C5D46
S1234BC0954040F48091EA0381FF04C081E08093A60402C01092A6048091B0079091B107B9
S1234BE090938B0080938A0080918A0090918B00909325068093240680919A07813021F020
S1234C0080919A07833011F481E009C080919A07843021F080919A07823029F482E080938F
S1234C20BC071092A50484E090E07FC08091B0079091B1078B5B9F4FE4F11092A50484E650
S1234C4090E090938B0080938A00909325068093240680919A07813021F080919A07833031
S1234C6059F481E08093BC0780916D0790916E0793FD13C02D9811C080919A07843021F021
S1234C8080919A07823059F482E08093BC0780916D0790916E0793FF2C981092A50488E201
S1234CA090E0909328068093270684E18093D2034BC08091BA079091BB0790938B00809321
S1234CC08A0020912B0630912C068091B0079091B107820F931F90932506809324068091F1
S1234CE09A07813021F080919A07833041F480916D0790916E0793FF2D9881E00FC0809100
S1234D009A07843021F080919A07823049F480916D0790916E0793FF2C9882E08093A504F9
S1234D2084E18093D20384EB90E090932806809327060AC080912B0690912C068C509E4F8A
S1234D4090938B0080938A002A9A7894FF91EF91BF91AF919F918F917F916F915F914F9164
S1234D603F912F910F900FBE0F901F901895A0E0B0E0BC01CD0128E532E040E050E00E948C
S1234D808E2D28E037E040E050E00E94E02DC901089521EB30E0F90110821092B60010922D
S1234DA0B2001092B300A0E7B0E08C9183608C93209A219A219A209A289A299A299A289ABE
S1234DC0EFE6F0E080818D7F80838C918C7F8C9386E0F901808384E680932006089581307F
S1234DE099F4289A289A80912F01843021F4299A299A1092D4031092CE071092CD07109206
S1234E00D3031092B1000895823049F4299A299A1092CC071092CB071092D40315BC089583
S1234E201F920F920FB60F9211242F933F934F935F936F937F938F939F93AF93BF93EF939B
S1234E40FF93F8948091D303843019F481E00E94EF267894FF91EF91BF91AF919F918F9174
S1234E607F916F915F914F913F912F910F900FBE0F901F9018950F931F938091EC039091E2
S1234E80ED030A9714F487E003C08091640486E08093B1001092B200809151049091520477
S1234EA0845F914018F41092B90716C080915104909152048D56974020F08EE08093B9070E
S1234EC00BC0809151049091520464E670E00E94B92D65506093B907E091B907F0E0E15169
S1234EE0FE4F80818093130180916404882329F02091CE048091180109C0E0915504F0913B
S1234F005604E654FB4F808120911801829FC00111249093AB048093AA04809151049091B3
S1234F205204825C914060F5809100019091010182FF1CC08091AA049091AB042091190127
S1234F4030911A01820F931F9093AB048093AA0480916D0790916E07846090936E078093F1
S1234F606D0780911B018093A90444C080916D0790916E078B7F90936E0780936D073AC08A
S1234F8080916D0790916E078B7F90936E0780936D078091A904823068F18091A904815071
S1234FA08093A9042091AA043091AB044091190150911A01E0911901F0911A0180911B0123
S1234FC07091A90460911B01240F351F90E0871B9109AC014E9FC0014F9F900D5E9F900D5F
S1234FE0112470E00E94B92D261B370B3093AB042093AA0480916404882309F0E8C0809174
S1235000C00787FD3FC08091C0078331DCF5E0915504F0915604E554FB4F4081E091550432
S1235020F0915604E654FB4F20810091AA041091AB04309194078091C007E091180150E0EF
S1235040421B510926EF8202C0011124830F911D9C01429FC001439F900D529F900D112445
S12350606AE070E00E94CD2DF0E06E9FC0016F9F900D7E9F900D1124800F911F9093AB04AD
S12350808093AA048091960787FD3FC0809196078F30DCF5E0915504F0915604E253FB4FB8
S12350A04081E0915504F0915604E654FB4F20810091AA041091AB043091BD07809196079F
S12350C0E091180150E0421B510926EF8202C0011124830F911D9C01429FC001439F900DCE
S12350E0529F900D11246AE070E00E94CD2DF0E06E9FC0016F9F900D7E9F900D1124800FEC
S1235100911F9093AB048093AA04809100019091010184FF5CC020911804309119048091B8
S1235120F8039091F90328173907FCF48091F8039091F9032091180430911904821B930BD5
S123514064E070E00E94CD2D80915704861710F460935704809157048A3018F089E0809316
S12351605704809128018093AC043091AC043430C8F08091AA049091AB04E0915704F0E01B
S1235180EB51FE4F2081820F911D9093AB048093AA0431503093AC0480916D0790916E0700
S12351A0806109C0109257041092AC0480916D0790916E078F7E90936E0780936D0780919A
S12351C0F8039091F9039093190480931804809100019091010191FD09C08091EA0386FF35
S12351E094C080916404882309F48FC0809122068F5F809322069091220680912306981753
S123520008F486C0109222068091F4039091F503E0919607FF27E7FDF095E050FA4F2081A6
S123522030E02817390734F48091200690912106890F19C08091F4039091F503E091960794
S1235240FF27E7FDF095E050FA4F208130E0821793075CF48091200618163CF48091200642
S123526090912106891B8093200680916D0790916E079D7F90936E0780936D0720912006D8
S1235280E0919607FF27E7FDF095E050FA4F8089332727FD309590E08C599F4F8217930732
S12352A054F4E0919607FF27E7FDF095E050FA4F80898C591EC020912006E0919607FF27B5
S12352C0E7FDF095E050FA4F4089332727FD309584E690E0841B910928173907CCF4E09119
S12352E09607FF27E7FDF095E050FA4F908984E6891B8093200680916D0790916E07926098
S123530090936E0780936D0703C084E6809320068091AA049091AB042091930730E062E0D8
S123532070E00E94CD2D269FC001279F900D369F900D112464E670E00E94B92D660F771FC0
S12353407093AB046093AA0480911E01209102043091030490E0C196821793070CF451C03C
S1235360809100019091010181FF4BC08091020490910304C397F4F020911C0130911D013F
S123538040911C0150911D01809102049091030460911E0170E06E5C7F4FFC01E49FC001A4
S12353A0E59F900DF49F900D11240E94B92D261B30E004C020911C0130911D018091AA045A
S12353C09091AB04280F391F3093AB042093AA04309B05C0809123019091240104C08091B7
S12353E01F0190912001909322018093210180916D0790916E07826090936E0780936D07B0
S123540011C080916D0790916E078D7F90936E0780936D0780911F019091200190932201B8
S1235420809321018091FA059091FB0583FF1CC0E091AA04F091AB0420913D018091AA04A7
S12354409091AB0464E170E00E94CD2D30E0629FC001639F900D729F900D11248E0F9F1F98
S12354609093AB048093AA04809100019091010190FF4DC08091EC039091ED038238910563
S12354800CF045C08091AA049091AB0420912A01820F911D9093AB048093AA04E091EC036A
S12354A0F091ED036091180120912A0182E890E08E1B9F0B70E0AB01849FB001859F700DF3
S12354C0949F700D11248FEF90E0FB01E89FB001E99F700DF89F700D1124882777FD80953B
S12354E0982F30E040E050E00E948E2D20E43FE140E050E00E94E02DC9012091AA04309117
S1235500AB04280F391F3093AB042093AA042091AA043091AB048091180145EF849FC00165
S123552011248217930754F480911801849FC00111249093AB048093AA040BC08091AA0457
S12355409091AB041816190624F01092AB041092AA048091AA049091AB0490935904809353
S1235560580478941F910F9108951F920F920FB60F9211242F933F934F935F936F937F9369
S12355808F939F93AF93BF93EF93FF93F8942091D303223039F0243009F44FC0213009F0D3
S12355A051C01CC08091CD079091CE078F3F9105D1F1C8F18091CD079091CE078F5F809364
S12355C0B3008091CD079091CE078F5F90409093CE078093CD072093D30334C00E943B271B
S12355E080915804909159049093CE078093CD078091CD079091CE078F3F9105A1F098F085
S12356008091CD079091CE078F5F8093B3008091CD079091CE078F5F90409093CE07809353
S1235620CD0782E007C08091CD079091CE078093B30084E08093D30305C081E00E94EF269E
S12356401092D3037894FF91EF91BF91AF919F918F917F916F915F914F913F912F910F90C3
S12356600FBE0F901F9018951F920F920FB60F9211242F933F934F935F936F937F938F93D3
S12356809F93AF93BF93EF93FF93F8942091D403223039F0243009F453C0213009F053C0DC
S12356A020C08091CB079091CC078F3F910591F088F08091CB079091CC078F5F87BD8091B8
S12356C0CB079091CC078F5F90409093CC078093CB0733C08091CB079091CC0787BD84E0F5
S12356E024C080915804909159049093CC078093CB0724E025BD16BC8091CB079091CC076D
S12357008F3F9105A9F0A0F08091CB079091CC078F5F87BD8091CB079091CC078F5F90405A
S12357209093CC078093CB0782E08093D4030BC08091CB079091CC0787BD2093D40303C00B
S123574082E00E94EF267894FF91EF91BF91AF919F918F917F916F915F914F913F912F91C0
S12357600F900FBE0F901F9018951F920F920FB60F9211242F933F934F935F936F937F9355
S12357808F939F93AF93BF93EF93FF93F8948091D403843019F482E00E94EF267894FF911F
S12357A0EF91BF91AF919F918F917F916F915F914F913F912F910F900FBE0F901F901895AE
S12357C0549A559A5C9A5D9A15BCEEE6F0E080818360808384E085BD16BC82E187BD0895E3
S12357E011B88FEF84B915B887B98AB9089588E98093C1001092C50083E18093C40086E1E6
S123580098E09093D4078093D3079093D0078093CF0786ED97E09093D2078093D10790934A
S12358205708809356081092D5071092290608951F920F920FB60F9211248F939F93EF93E5
S1235840FF938091D507882311F1E091D307F091D40781918093C600F093D407E093D307DB
S1235860E655F84030F086E198E09093D4078093D3078091D50781508093D5078091D5072D
S1235880882329F48091C1008F7D8093C100FF91EF919F918F910F900FBE0F901F901895C3
S12358A01F920F920FB60F9211242F938F939F93EF93FF938091C600E0915608F091570847
S12358C08083809129068F5F80932906809156089091570801969093570880935608865101
S12358E0984030F086ED97E09093570880935608FF91EF919F918F912F910F900FBE0F90A4
S12359001F90189580912906882319F42FEF3FEF1AC0F89480912906815080932906E091B9
S1235920D107F091D2072191F093D207E093D107E651F84030F086ED97E09093D207809350
S1235940D107789430E0C9010895982F8091D5078F33E0F78091D507803410F080E00895FD
S1235960F8948091D5078F5F8093D507E091CF07F091D00790838091CF079091D0070196A5
S12359809093D0078093CF078655984030F086E198E09093D0078093CF078091C1008062D7
S12359A08093C100789481E00895CF93DF93EC0104C00E94A52C8111219688818823C9F750
S12359C081E0DF91CF91089585ED93E00E94D52C08958DED93E00E94D52C08958091290663
S12359E008959F92AF92BF92CF92DF92EF92FF920F931F93DF93CF93CDB7DEB729970FB699
S1235A00F894DEBF0FBECDBF7C01062FDE011196E0EEF3E089E001900D928150E1F719E0EC
S1235A2099E0A92EB12C6E010894C11CD11C8CE2982E002371F09501211B3109802F90E07D
S1235A402817390730F01150F601E10FF11D908200E01150F601E10FF11DC7016AE070E0A3
S1235A600E94B92D805D8083C7016AE070E00E94B92D7B016115710511F4002311F0063009
S1235A80C0F219E0141B7E010894E11CF11C07C0F701E10FF11D80810E94A52C1F5F19300B
S1235AA0B8F329960FB6F894DEBF0FBECDBFCF91DF911F910F91FF90EF90DF90CF90BF90E6
S1235AC0AF909F900895DF92EF92FF920F931F937B018C01FB010995D82EC8010196F701DF
S1235AE00995982F8D2D1F910F91FF90EF90DF900895DF92EF92FF920F931F93D72E7A01C2
S1235B008C01FA010995C80101966D2DF70109951F910F91FF90EF90DF900895629FD0018F
S1235B20739FF001829FE00DF11D649FE00DF11D929FF00D839FF00D749FF00D659FF00DE6
S1235B409927729FB00DE11DF91F639FB00DE11DF91FBD01CF0111240895991B79E004C097
S1235B60991F961708F0961B881F7A95C9F780950895AA1BBB1B51E107C0AA1FBB1FA617F7
S1235B80B70710F0A61BB70B881F991F5A95A9F780959095BC01CD01089597FB092E07267A
S1235BA00AD077FD04D0E5DF06D000201AF4709561957F4F0895F6F7909581959F4F0895DE
S1235BC0A1E21A2EAA1BBB1BFD010DC0AA1FBB1FEE1FFF1FA217B307E407F50720F0A21B9B
S1235BE0B30BE40BF50B661F771F881F991F1A9469F760957095809590959B01AC01BD0131
S1235C00CF01089597FB092E05260ED057FD04D0D7DF0AD0001C38F450954095309521950C
S1235C203F4F4F4F5F4F0895F6F790958095709561957F4F8F4F9F4F0895F894FFCF2F0007
S1235C40010002000300040005000600070008003228E80390010614001E1E003C581B58E9
S1235C601B88136419121E01010203040A0411C4098813C4096400DCE64003020A1432465D
S1235C80962800000000000000000000000000000000000000000000000000000000000042
S1235CA00000000000000000000000000000000000000000000000000000000000000000E0
S1235CC00000000102030405060708090A0B0C0D0E0F100102030405060708090A0B0C0DDD
S1235CE00E0F100102030405060708090A0B0C0D0E0F1014161718191A1B1C1D1E1F20218D
S1235D00222324191A1B1C1D1E1F2021222324252627271E1F2022232425262728292A2B31
S1235D202C2D2E000204060708090A0C0E28262422201E1E1E1E1E1E1E1E1E1E1EF0FF8023
S1235D40BBE0880465484BA438022BF0207019CC13860F440CC209D0074C061B052A046A0E
S1235D6003D1025602F201A1015F012801FB00D600B7009D0087007500660059004D004462
S1235D80003C0034002E0029002500F0FF80BBE0880465484BA438022BF0207019CC13867E
S1235DA00F440CC209D0074C061B052A046A03D1025602F201A1015F012801FB00D600B700
S1235DC0009D0087007500660059004D0044003C0034002E0029002500F0FF80BBE0880454
S1235DE065484BA438022BF0207019CC13860F440CC209D0074C061B052A046A03D1025669
S1235E0002F201A1015F012801FB00D600B7009D0087007500660059004D0044003C00347D
S1235E20002E0029002500F0FF80BBE0880465484BA438022BF0207019CC13860F440CC22C
S1235E4009D0074C061B052A046A03D1025602F201A1015F012801FB00D600B7009D00875C
S1235E60007500660059004D0044003C0034002E00290025000000F5047E05AE066C08C009
S1235E800AB30D630F8B10D7118813000000000A000F001E003C007800FA007201E00180EB
S1235EA0028002000008000A000C000E00C80A4A067E048403AC0D641A0020002700320053
S1235EC03E0066008E00B202EB02240337034B03560361037003E800D600C200B0009D003F
S1235EE08A00780078006500520040002D001900070000000100010001175A5A5A505050C8
S1235F00505050505050505050500A00030000FA3204041B5B481B5B324A000D0A00202015
S10B5F20202020202020200095
S50302FA00
